:0200000480007A
:100000006F00C004732F2034930F8000630AFF0336
:10001000930F90006306FF03930FB0006302FF038A
:10002000170F0080130F0FFE63040F0067000F000F
:10003000732F203463540F006F00400093E19153FD
:10004000171F000023203FFC6FF09FFF930000006C
:10005000130100009301000013020000930200004E
:100060001303000093030000130400009304000036
:10007000130500009305000013060000930600001E
:100080001307000093070000130800009308000006
:100090001309000093090000130A0000930A0000EE
:1000A000130B0000930B0000130C0000930C0000D6
:1000B000130D0000930D0000130E0000930E0000BE
:1000C000130F0000930F0000732540F1631005002B
:1000D000970200009382020173905230735000180F
:1000E000970200009382020273905230B7020080A0
:1000F0009382F2FF7390023B9302F0017390023AF5
:100100007350403097020000938242017390523046
:10011000735020307350303093010000970200007C
:10012000938282EE73905230130510001315F5017F
:10013000634C05000F00F00F930110009308D005E9
:10014000130500007300000097020080938282EB89
:10015000638A020073905210B7B20000938292102B
:100160007390223073500030372500007320053023
:100170007350300097020000938242017390123452
:10018000732540F173002030370580FF530505F0DB
:10019000531505E093031000930120006316750EBC
:1001A000370580BF530505F0531505E09303200084
:1001B00093013000631A750C370580801305F5FF35
:1001C000530505F0531505E09303400093014000EB
:1001D000631C750A37050080530505F0531505E0CB
:1001E00093038000930150006310750A130500000B
:1001F000530505F0531505E09303000193016000DA
:1002000063147508370580001305F5FF530505F0E5
:10021000531505E093030002930170006316750601
:100220003705803F530505F0531505E0930300049F
:1002300093018000631A75043705807F530505F02C
:10024000531505E09303000893019000631E7502A7
:100250003705807F13051500530505F0531505E09C
:10026000930300109301A000631075023705C07F4F
:10027000530505F0531505E0930300209301B000EA
:1002800063147500631030020F00F00F63800100EB
:100290009391110093E111009308D005138501009B
:1002A000730000000F00F00F930110009308D005B9
:1002B0001305000073000000731000C00000000070
:0402C000000000003A
:1010000000000000000000000000000000000000E0
:1010100000000000000000000000000000000000D0
:1010200000000000000000000000000000000000C0
:1010300000000000000000000000000000000000B0
:081040000000000000000000A8
:040000058000000077
:00000001FF
